:020000040000FA
:04000000A6EF00F077
:06002A00640EF66E010EEB
:10003000F76E000EF86E0900F550056E0900F550D8
:10004000066E055002E106503BE00900F550006ED7
:100050000900F550016E0900F550026E0900090013
:10006000F550E96E0900F550EA6E09000900090033
:10007000F550036E0900F550046E09000900F6CF33
:1000800007F0F7CF08F0F8CF09F000C0F6FF01C085
:10009000F7FF02C0F8FF035002E1045007E0090037
:1000A000F550EE6E0306F8E20406F9D707C0F6FF36
:1000B00008C0F7FF09C0F8FF0506C4E20606C5D769
:1000C0001200D9CFE5FFE1CFD9FF00C0E5FF01C0A5
:1000D000E5FF02C0E5FF03C0E5FF020EDBCF00F045
:1000E000030EDBCF01F000C002F001C003F0FF0EF1
:1000F0000026D8A001060250031006E0FA0E026E98
:100100000000022EFDD7EFD7E4CF03F0E4CF02F0DA
:10011000E4CF01F0E4CF00F0E4CFD9FF1200620E8B
:10012000D36E0F0E936E816A006A100E005CFCE2C3
:100130000038F00B816E000EE56E640EE56E61EC2A
:1001400000F0020EE126002AF0D7120012EEFFF0B6
:1001500022EEFFF0F86AA68EA69C15EC00F08FEC5C
:1001600000F0FFD7010072010000800000000100D4
:04017000000000008B
:00000001FF
